:1000000002780030B402D25202168F758C10D26B77
:1000100002155730B502D25102171E32FFFFFFFF03
:10002000FFFFFF32FFFF020032FFFF353444555619
:1000300020208520F0E4787FF6D8FD85F02090E838
:1000400000E4F0A374EFB583F874F0B582F3A20373
:10005000920190006D75A0C078007402F208E493DC
:10006000F2A308046023E493F2A30880ED15491479
:1000700000255D0638073C094622890FC21D301D48
:100080001020AD0A8C0A7DFFFFC20430961D309708
:100090001A7C14C296209713D29630970EC29720DE
:1000A0009609D297309604DCEAD204D296D2977D94
:1000B000177C4C0D90412D75A0807800E493F2A33D
:1000C00008B8000205A0DCF4DDF27583F41280604C
:1000D00090F408787775F003128079D200743F129B
:1000E000412C90E7FE12412C4017F0A3B4030040CE
:1000F0001212412C400BF0A312412C4004F0A380BB
:1001000002C20012412C745412412C1225EE122D01
:10011000607435122D79121A3C50726F6772616DDE
:1001200020636865636B73756D202D2D2D2D200068
:10013000E4FBFF900000C3742D24B4FC7441341B15
:1001400004FDBC00011DE4932BFBE43FFFA3DCF6A0
:10015000DDF4A3A3E4932B7006A3E4932F600B12AA
:100160002D6B12209C7590FD80FE12209130003383
:10017000121A3C4F7665726C6179207265766973EC
:10018000696F6E202D2D2D2D20200090E7FEE0249C
:1001900030A3121A77E02430A3121A77E0121A77EC
:1001A0001220A67583F01280607583F4128060902F
:1001B000F418788875F003128079745A12228974C1
:1001C0001BFD12228974B4FC12228990412D0DE48A
:1001D00093122289A3DCF8DDF6E493A3122289E4CA
:1001E00093A312228974A13002027461FE7C00790B
:1001F000401222891202251222A7F7543F09500A01
:10020000F8EEC4440F68D36001C3EC92E303FC0E24
:10021000EE30E2DD90021DEC93F5778011030700CC
:100220000B0000000F7B127A00DAFEDBFC22121AB0
:100230003C546F74616C20706F72747320666F75BC
:100240006E64202D2D2D202000AD770D7A00120A2E
:10025000A11220A67436122D791209AFE577B404E5
:1002600000500302035824FD0303FCA20592F77912
:1002700040E70965F054806003757700DCF3121ADB
:100280003C536C61766520636F6D6D756E6963615B
:1002900074696F6E202D2000C3E5776006122091EF
:1002A00002035812209C7C017940121A3C20536CA6
:1002B00061766500AD047A00120AA1E76068F5F086
:1002C000121A3C2020526F6D3A2000A2F012034413
:1002D000121A3C202052616D3A2000A2F112034410
:1002E000121A3C2020492F4F3A2000A2F212034458
:1002F000121A3C202050676D3A2000A2F3120344EA
:10030000121A3C2020547970653A200020F70B1215
:100310001A3C4D554C544900801D121A3C50432F35
:100320004D4143008011121A3C20204E6F2072650F
:1003300073706F6E7365001220A6090CBC040280F6
:10034000170202AA4009121A3C424144200022121C
:100350001A3C474F4F440022E5777008122D727502
:1003600090FE80FE90E865F07437122D791209AF87
:0E0370003003081230A7500302040675A0E9FE
:10037E0079009064007D017C507F007B00E493F354
:10038E00120416A309B9000205A0DCF1DDEF75A079
:10039E00EA79009065007C00E493F579E493F3121A
:1003AE000416A309DCF6121A3C436F6E66696720C9
:1003BE00636865636B73756D20202D2D2D2D2000C8
:1003CE009067FEE4932B7027A3E4932F702190E99E
:1003DE0000E0B4011A90E901E0B4231390E902E0C1
:1003EE00B4010C90E903E0B40405122091803012A0
:1003FE00209C7590FF122D861207E84006122D9054
:10040E0002037B122D9780ED2BFBE43FFF2201238D
:10041E0001040005100F2B78101A00002100009027
:10042E00E904E0A2E09238A2E1922490E905E0907E
:10043E00E86EF0A3F090E906E090E86CF0A3F0907F
:10044E00E907E0F57790E908E090E863F090E909B4
:10045E00E090E86AF0A3F090E90AE090E868F0A373
:10046E00F090E90BE0F55F90E90CE0F57690E90D80
:10047E00E0F57890E866F090E90EE090ED00F0304F
:10048E00020990E865E0F57F022615128011538966
:10049E00F0438901D28CD2A9D2AF755160755060EC
:1004AE00755A40755940120638306E1F74201285E9
:1004BE0052121A3C5043206B6579626F6172642050
:1004CE0064657465637465640D0A001207961207FD
:1004DE003C303908121AFA755F12803330251F121C
:1004EE001A2A0D0A00121A3C50532F32206D6F75C6
:1004FE0073652064657465637465640D0A00206E0F
:10050E00031206A0306E05121FB5C25C1280EA12ED
:10051E0009B8D268D26E757B00757C0090E857746E
:10052E0006F090E8507400F0A3F0122DA1120A34D8
:10053E002001030205F9121A3C0D0A5072657373FD
:10054E00200090059E122D069005B4122D06200354
:10055E00581205671205758056121A2A656E746553
:10056E0072206B65790022121A58656E74657220BE
:10057E006F6E206B657970616400223098FDC298B1
:10058E00E599221230A7400122B40702D322C322DA
:10059E00C048697420656E74657220746F20707225
:1005AE006F6365656400932000120567120575126E
:1005BE001A3C20746F20636F6E74696E75650D0A38
:1005CE0000E412412C4390032003121205914009BE
:1005DE003098F8120589B40DF2D2D1800E12059121
:1005EE0040093098F8120589B40DF2437DC3C20359
:1005FE00E412412C12412CA25D924AC25D12178068
:10060E00A24A925D128520B3921B122CF220001585
:10061E00121A3C0D0A5374617274696E67206D6113
:10062E00696E0D0A00C201020AC9C2A8D21F90E863
:10063E008574FAF0E55F540FB40548C2AA1207B1EB
:10064E00C2B2120225D2B3780F1285C17C051202F6
:10065E0025DCFBC2F090F401E030E02654E0790096
:10066E00600279FF5382F8438203E0B900E720F07D
:10067E000AB4FEE1128EE9D2F080DA90ED00F012AB
:10068E00853422B40408C2AA1240B1D2B322120792
:10069E008322206E7575B0FF7A0A7914E5B0543C4A
:1006AE00F8E5B0543C687009D9F7E8542464246026
:1006BE000CDAE9121A3C0D0A50430080537850D8D8
:1006CE00FE7904B2B27850D8FEA2B413A2B513D9F3
:1006DE00F2D2B2B4CC14755F4412063812073C1233
:0E06EE001A3C4170706C65008026B488028052
:1006FC0003B4DD18755F5512063812073C121A2A1E
:10070C000D0A00121A3C53756E008006121A3C50EA
:10071C004300121A3C206B6579626F61726420632E
:10072C0061626C6520646574656374656420002285
:10073C00C225C24DE55FB455061207B1C2AA22B458
:10074C004403C2AA22C24B1207B11209AF121AAA51
:10075C00121FF530390122202514304B19E55F5456
:10076C00F0B4500122E55F540F4420F55F22E55FA1
:10077C00540F4410F55F22752508D288D2A8C2897F
:10078C00D2B2121F784002D26E22752608D2BAD28B
:10079C008AC28BD2AAD2B31209AF121F954005D2CE
:1007AC0025121F9522E55FC4540775F000B40304AD
:1007BC00D2F08005B40502D2F07866C2F190F40054
:1007CC0012807990F4101280791207D922D2EEF1AE
:1007DC00DFC2EE79007A40D9FEDAFC22121A3C52C2
:1007EC00656C6F6164696E67204E5672616D207422
:1007FC006F20666163746F72792064656661756CD5
:10080C00740D0A00122DB91209467B007F0075A0E9
:10081C00EB790090041C7C00E4BC5000502EBC40D2
:10082C0000400890412CEC540F801BBC300040045D
:10083C0074108018BC200040047401800FBC1000A0
:10084C0040047402800693BC0702E577F312041689
:10085C00A3090CBC00C29064001208D6500122906F
:10086C00EB007C007412F0120416A3DCF790650008
:10087C001208D650012290EB007C40E4F0A3DCFB84
:10088C007E08906600BE010E75A0EB793EC3E49B1A
:10089C00F309C3E49FF375A0EB79001215495002DC
:1008AC00D322DEE17B017E40906800C082C083C011
:1008BC00061208FED006D083D08275A0EB79001208
:1008CC0015495002D322DEE3C3227C0075A0EB79DC
:1008DC0000EC2582F582EC29F9C004C082C0831299
:1008EC001549D083D082D0044007EC2440FC70DC46
:1008FC00C322780490EB00D2217C00EC242B83F0F3
:10090C00BC081CBB00067D007A0180048B057A00B4
:10091C00C000C0061220ADD006D0007C0B8002A314
:10092C000CBC10D70BD8D2C22122436F6D707574DA
:10093C006572202020202020202090095E75A0EFD9
:10094C007980E493F3A3097409B583F674AFB58287
:10095C00F122C083C08290555574AAF0902AAA74D3
:10096C0055F090555574A0F0D082D083C083C082CE
:10097C00C0017C40E3F0DC02800409A380F6C3F8DC
:10098C00E49368400430E7F8D320E7F4D001D08238
:10099C00D0837C40E493F8E3A309B50004DCF5C3F1
:1009AC0022D32278007900D9FED8FC2274E61222D8
:1009BC00897C01EC12228990ED00E0A3122289DCE3
:1009CC00F990E9147E04120A2590E9247E14120A87
:1009DC002590EA047E24E578603790E930E0FA85CA
:1009EC0078F0A42404C39578F5827583EA7C0C799D
:1009FC0005EE1222890EE578B501005005E07A016A
:100A0C0080027412122289E5822AF58209DCE280C6
:100A1C0003120A25E4122289227C0CEE1222890E82
:100A2C00E0A3122289DCF422E578B40200402E7C8B
:100A3C0001BC0400C00450098C74741612813B80F4
:100A4C00147401122208ECC412220874EF1222084A
:100A5C007416122208E578D0040CB504D422C0E038
:0E0A6C00C082758205E4D5E0FDD582F9D08206
:100A7A00D0E02275F010A42400F582E5F03468F580
:100A8A008322120A7D5382C075A0EB79007C40E470
:100A9A0093F3A309DCF922300124D22190E810C093
:100AAA0004C0011220ADC2217C0390E810E0128537
:100ABA005230000312412CA3DCF3D001D0042230BF
:100ACA006B0312156AE55C7013304C05121FB5C230
:100ADA004C306D0812073C128E7EC26D122DE690C4
:100AEA00E866E0F578E55F540FB40416D55B347513
:100AFA005B10E5537003123F04E55C7026123F60F9
:100B0A008021B40508121A84121AAA8016C24B2030
:100B1A003911121AAA304B0BE55F54F0B420005079
:100B2A0002D26D205E0C20700C207109206F060223
:100B3A000B84020D8DE55C6015207209D27290E873
:100B4A003FE4F0803590E83FE0B40200402C7D039A
:100B5A00C27230251574F5121F07206707121F95F8
:100B6A0040028006DDEAC225C24DD27F752608857D
:100B7A00595A755C00D25F12178030195C1222A78D
:100B8A005057F8128EC6120B95804E30E73AB48051
:100B9A0008D268747E1285522230E6175300071273
:100BAA000FC25407B40400502FE054F048F0F5790E
:100BBA00D25D2230E505A2E0921B2230E41AD25C13
:100BCA00128EA9E8540FF0227583E8E575C4540F14
:100BDA004440F582E8F0D2752212864D4003020E97
:100BEA0029307A03020C8C30272B90E850E0F8A3C6
:100BFA00E0C868601E75A0ECE2F556700908B8C036
:100C0A00027800E2F557D27A08B8C0027800E8F014
:100C1A00020C8CC22720766AE550B551028063E542
:100C2A005FB444028022B45502801DA851E6B4F78D
:100C3A0006D211D2148007B4F80EC211D214E551AB
:100C4A0004546FF551020D8D121ACC30010F307A0F
:100C5A000CE556128F0C7005E557128534102302E5
:100C6A008020E550B5510280F91210A2128ED002EE
:100C7A002114E550B5510280F91210A2128ED50244
:100C8A0021CF307B1112412C207B083054051214DD
:100C9A0000C254020D8D202747207C03020CB1129A
:100CAA002DF2403C020D8D203936307A33E556B4A8
:100CBA004A04D263802AB4CA1230631BE55F540F18
:100CCA00B40504D2538019D2768015B42D09305355
:100CDA0006D276C2538009E4F57A522CC25EC25318
:100CEA00301907307A32C27A805BE5537050307A15
:100CFA0027C27AE55654FCB428258556F090E82098
:100D0A0075552030F10574E0120D2430F00574F0A9
:100D1A00120D24E557120D248069F0A305532230E1
:100D2A001810E556700CE557B41900400512813BBE
:100D3A008045128B35E553603E755520C27A75A001
:100D4A00E8A855E2F830192A122252E556128EC145
:100D5A007001F4122289B4FF08E557A21892E680BE
:100D6A0009E55654FCB4280FE557128EBC122289A5
:100D7A0080051281C2400C307609E5537005C276AF
:100D8A0002100A307302802BE559B55A02802412E8
:100D9A001D4830011E30731B74201285527475125F
:100DAA00855290E82DE0128534A3E0128534A3E041
:100DBA00128534E55C700F307365128CEAE55C606D
:100DCA005E755E28C27375A0E8A95EE3F830194C17
:100DDA0012225290F41A7415F07582187407F09062
:0E0DEA00E828E0128ECB1222891222525015F8
:100DF800B480127C0390E829E0A3128ECB122289DA
:100E0800DCF6755C0090F419E030E3FC30E2F99010
:100E1800F41A7415F07582187403F0020E29128200
:100E28001F12814C304F07302622C226C24F105A5B
:100E38004010592A10584F203D54105D75103C0F32
:100E4800105C0F105B12105F12107509020FB702C9
:100E58000ED0020F29020F77020EEE020EF8128E44
:100E6800A95407303905A21BB392E7120F11020FDC
:100E7800B7120FD6203905B40302D23CA23992E743
:100E8800120F11020FB7E576120F11020FB790E893
:100E980077E004F0A2E01403C2E7900FCD93600856
:100EA8004002800874FC8004C23D74F4120F1102E1
:100EB8000FB7203909E55F5407B40400500774F0F0
:100EC800120F11D25A020FB7E579540FB4040280F9
:100ED80003B4050474F88009D23D90E877E4F0740F
:100EE800FAF111020FB774F1120F11D258020FB7AD
:100EF80030251385595A12207374F4121F0720677E
:100F080005121F95C27F020FB7C2267905C0E012ED
:100F18001EB0D0E0306605303902D9F1D24FD26A1E
:100F280022128EA9F8E55F540FB40407E81240FEB8
:100F3800020FB7B40525C000780E1285C1D000E8AD
:100F4800A2E092F2A2E192F0A2E292F3A2E392F17D
:100F580053F00FA8F01285C1020FB77D0A74ED1285
:100F68000F11303905306602DDF3D259020FB7751B
:100F780083E8E575C4540F4440F582E0F8E55F5412
:100F88000FF9E579540FB404028024B40512B80EA1
:100F980003020F29203912B90515E81285C1800FFF
:100FA800B8ED03020F29B9ED06E8120F118000C24F
:100FB80075205E03020AC902101A7583EAE57644B1
:100FC80000F582E022391911125914765800E57992
:100FD80054077802B4030040027803E55F54FC45E7
:100FE80000F55F30391AE579D2F054F06002C2F0AA
:100FF800E57954077803B404005005A2F092E4227E
:10100800E82290E873E551F0757E00D25E90E8849E
:10101800E4F090E884E0B42003021145C3E55024CD
:10102800109551540FF8E55F540FB4041BB8020033
:1010380040591210A2FE1210A230E74CCE20E74809
:1010480053067F6E7042803BB405234021B80300ED
:1010580040391210A2FE1210A230E72CCE20E72849
:1010680053067F6E70221210A2B47F1C8015B8033D
:101078000040181210A2FE1210A2B4F00B1210A217
:101088006E70051210AF704C02114EE86009A8513D
:1010980086061210AF60F1020AC9A851E6128EE462
:1010A8000853006F885122EE121ACF307A1DC27A87
:1010B8009011A27C008002A30CE4936016B556F749
:1010C8009011C3EC93B43105200008E422500420A9
:1010D80000F91422BC0A005036E57E75F00AA42CEB
:1010E800500205F0F57E85F07FE52C5407701D054C
:1010F8007AE57AB4020AE577B46300500F02116109
:1011080050FBE577B409005003021161021015BCC9
:101118001100500874F72C422C0210159011E3ECC2
:1011280024F6230493C0E0EC24F62393C0E022C302
:1011380078007908102605D8FBD9F9D322E52C5474
:1011480007700302116190E873E0F551755800E4E7
:10115800F57A522CC25E020D8D12117F4016F57E73
:0E116800E577B57E00400D857E76C238C270F8
:10117600D26FC25DC25C020CE1857FF0E5F0B4027D
:1011860000500CE57E20F005600514C32260FBD3F9
:10119600224410F0A3F0A3EEF0A3F0223031323354
:1011A6003435363738397674706D61777573786B88
:1011B600473B3A43726E69642E0C620F003232323C
:1011C6003232323232323232303030303030323205
:1011D60032323232323232323131323232120F124E
:1011E600141221127A1230124D12611325132A138A
:1011F600FA1345132F1339133D135413BE13AB13B0
:101206008E138413711394139990E868800390E801
:101216006CE57FAE7E121197020CE112117F4051F0
:10122600604FF577121780020CE1E57F7043E57E8B
:10123600B48000503CC082C08390E863F0D083D075
:1012460082121FE2020CE1E57F7026E57EB4020001
:10125600401F90E930F0D26F020CE1E57F7012E595
:101266007EB41100500BF57890E866F0D26F020C50
:10127600E102114EE57F701FAA7EE57E6019B40B70
:1012860000403EB41400400FB41600400DB41E00DA
:101296004005B421004014020CE1E57EA2E0E55FC2
:1012A600C2E392E3F55FD26D020CE1E55F540FF9FC
:1012B600E57E24EB834501F55FD26D020CE110203B
:1012C60050120FC2BA04047444803EBA0504745521
:1012D6008037BA0B0474668030BA0C0474778029A0
:1012E600BA04004013540FCA24FBB40404740580E6
:1012F60016B405137400800FC4540FA87953000761
:10130600B8040040027401C44AF579D25D120FC2D6
:10131600E579F0FBD24AE582FE122575020CE1D290
:1013260038020CE1C238020CE1D270C238C25DC28A
:101336005C8009D27180F4A201B39201020CE1E54E
:101346002C540760062409FC0211240211612000B6
:10135600031225E81219DCC238E55FB4440280DCCA
:10136600B4550280D7D24CD26D80D130000AD27CDF
:10137600D27B12412C020CE1122EED020CE1D27B43
:10138600C27C12412C020CE112412C020CE1B22467
:10139600020CE1E579B4550A7400121D30741E1270
:1013A6001D30020CE17E0090260FEE936007FA12C4
:1013B6001D100E80F2020CE11213C4020CE1E57955
:1013C600540FB40400501120180F201921E574D2CF
:1013D600E212847BE41284B522E57412847B74EFF6
:1013E6001284A4E57412847B74311284A4227431AD
:1013F6001222082212140002134212140912147A3D
:10140600500022E578606C7B00EB12847BC023C21F
:101416001974EF1284A4EB12847B74151284B5D070
:10142600230BBB04028006E578B503DD22E57824AC
:10143600FC6040FB757540D219D21874011222085F
:10144600E575122208D2237415122208E5752410B8
:10145600F575120A6ADBE4741612220812180512D0
:101466000A6A120A6A120A6A120A6A120A6A120ACE
:101476006AD26F2290E904E0A23820000292E0A22C
:101486002492E1F090E86EE090E905F090E86CE0D7
:1014960090E906F0E57790E907F090E863E090E9D7
:1014A60008F090E86AE090E909F090E868E090E9D1
:1014B6000AF0E55FB444028003B455047412800256
:1014C600C2E090E90BF0E57890E90DF090ED00E0D0
:1014D60090E90EF01209467B007F007C5090E900EF
:0E14E600E493120416A3DCF875A0EB790090D5
:1014F400EA007C00E493F3120416A309DCF690647A
:101504000075A0E9790012154950012290644075D4
:10151400A0E979401215495001229065001208D6BD
:1015240050012290EB007C40E4F0A3DCFB90EB3E06
:10153400C3E49BF0A3C3E49FF09067C075A0EB796C
:101544000012154922128A5112EF8092F0128A2653
:10155400A2F022202B06107E0375250820330610E6
:101564007D0375260832C26B303B12C3E55024104C
:101574009551540FB409005004D2B2C23B303A160C
:10158400C3E5592410955A540FB409005008D2B336
:10159400C23AD249802F90E876104927E004B40873
:1015A400004021755C00E55AB559028016F8E6B48E
:1015B400AA0E0853004FE6700785595AD26D80036E
:1015C40085595AE4F012412C106A11304F0EC24F63
:1015D400C259C25AC258C25CC25DC25B20393230A1
:1015E40079173077101218C9743112412C12412C1A
:1015F400C277122CF2C279801290E86912166650F2
:101604001012189FD27712412C800690E8681216A7
:101614005E90E884E004F090E83FE004F012855D19
:1016240020111F201A1C207B1930381690E86D12E7
:101634001666500ED215D270C25DC25C90E86C1270
:10164400165E303F1190E867E004F0B402004006F3
:101654001218FC122FC2122FCF22E0A3F0A3E0A392
:10166400F022E02410F0501FF84410F0A3A3E0B8D7
:101674000002601314F0B4FF09E81415821582F017
:10168400C3227003E86002C322D322202F1E302B12
:101694000A105206D279D27E152532C55203D2E7FA
:1016A400105202C2E7C5521525C22B3210285775B5
:1016B4002508105216D274C2B2C001C55264AA6081
:1016C40006C5527930803864AA80173013E7C2B255
:1016D400C001C55264FA7008D226C5527930801F01
:1016E40064FAC552A950A7520953016F8950C9041D
:1016F400546F65517006D23BC9D00132C97926D9DD
:10170400FED2B2D00132C552D21310520520D007F6
:10171400800330D002C213C5523220372030330C3C
:10172400105108D279D27DD249152632C55B03D235
:10173400E7105102C2E7C55B1526C23332103028C8
:1017440075260810510132306C31C001A959A75BCC
:101754000953014F8959C24BC904544F655A700447
:10176400C2B3D23AC9D00132C55BD26C1051052044
:10177400D007800330D002C26CC55B32205E2720C4
:101784005924205A2120581E203D1B205C18205D1E
:1017940015203C12205B0F10700D107118C26FE5FC
:1017A40077B57600501B220576E577B576005011A3
:1017B400757600800C1576E576047005857776805D
:1017C40000C20774AA42C0D21F1289ED12313A2016
:1017D400390312412C204E031218FC121805304E06
:1017E4000D121A2A2066702A00C218C21922121970
:1017F4007A12193512314110150122301402D25BCC
:1018040022A97612181CF575A2F69219A2F792185D
:10181400A2F5924E12869922203904E5787006E9E1
:10182400C454F0802EE578B40F03E980268578F05F
:1018340090E930E0A414B50100500BC304F5F0E9BD
:1018440095F0257880DA90E930E0F5F0E984540FDA
:10185400C445F0F875F00020390BE854F0C4B578AD
:0E186400005002D2F7E854C06002D2F6C0F085
:1018720090E930E08578F0A4C0E0E5F06006D0E0C1
:10188200D0F0E82290E865E0D0F025F0C39578B575
:1018920001005005D0F0D2F522D0F0E82220180540
:1018A20020191C801FE575C4540312847B74EF1247
:1018B20084A4E575C4540312847B74021284A47454
:1018C20002122208C2EC22201905201802802830B8
:1018D2001905740C12220830181FE575C45403123E
:1018E200847B74EF1284A4E575C4540312847B7460
:1018F2000C1284A4201902D2EC22C23F20191F30FC
:10190200182EE575C4540312847B74EF1284A4E587
:1019120075C4540312847B74161284A48012301886
:101922000A74EF1222087416122208741612220880
:10193200C2EC2220183C30192F74091222081222FC
:1019420067D268F854706020C4B40600501AE8A246
:10195200E7921B128EA9E8540FF0E8C45407F8125C
:101962000FC254F048F08003120FC2F579D25DD253
:101972005C22120FC2F5792220182320190EE57578
:10198200C45403F57444FCF590D2EC227401122283
:1019920008E57554F0122208740C1222082220194C
:1019A20024121980E57412847B74EF1284A4E57406
:1019B20012847B74011284A4E57412847BE575544D
:1019C2000F1284A42212198E74EF122208740112CB
:1019D2002208E575540F1222082220181020193A05
:1019E2009092A5E574540393457DF57D2230190349
:1019F200121A1CE574540312847B74EF1284A4E55A
:101A020074540312847B74301284A4E57454031258
:101A1200847BE575540F1284A4227430122208E5E7
:101A220075C4540F12220822D083D082E493128507
:101A320052A3E493B400F7740173D083D082C082BE
:101A4200C083E493128552A3E49370F8200007D078
:101A5200E0D0E0740173D083D082E493B40A0280B0
:101A62000D30010A300007C00112412CD001A3E45D
:101A72009370E90473300109128552300003124158
:101A82002C2290F401E030E01E54E07900600279EB
:101A9200FF5382F8438203E0B900E7A950F70550EB
:101AA20053506FD27980DB2290F411E030E01A5368
:101AB20082F8438203E0A959F7128F250559535939
:101AC2004FD24BD249D27980DF221210A2F8FCAE5B
:101AD2005F53060FBE0402804EBE05028049E558E0
:101AE2006003021C01B8AA06D26E121FB522B8DF2B
:101AF200004034B8EF16D223D239743012412C751B
:101B02007800C23875770FD26ED22522B8F00475EC
:101B1200580122B8E00475580222B8E1047558044D
:101B22002275F000021BD1E55F540FB40406902326
:101B3200CA021BC3B4052BE5795403B4031F90ED0D
:101B420000E0B433028016B434028011E8A2E792B6
:101B5200F0C2E7B458077420A2F0021BF790244A9F
:101B6200805FC392F0E55F54039022B77885B40397
:101B72000590233C788EECB50000505393A8792051
:101B8200393BB844028003B85533A85F53000FB8FD
:101B92000A00500CB44C02741BB44B21741E801DFD
:101BA20030241AB44C04744E8013B44D04744F8024
:101BB2000CB44E04744C8005B44F02744DA2F080F4
:101BC20006E8A2E7C2E79364FF701C92F0C2F1E557
:101BD2005F6479540360277428A2F092E0A2F19224
:0E1BE200E1F5568C57801264FF30E709755606
:101BF0000092E7F557800492E7F556D27A755800BF
:101C000022E558B401028012B40204C2F0800FB47D
:101C10000305D2F0021C26021CE6D3021B65E8B4C1
:101C2000F00475580322901C61E4A393A36015B5DA
:101C300000F7E49330F0022402F557755600D27A8B
:101C400075580022901C67D2F1787FECB5000050E7
:101C50008093F5567003021BD130F0034356800287
:101C60001BFB1201590200000000000000000000F0
:101C700000000000000000004D00004B00000000CC
:101C80000000000000004E000000000000004F00B7
:101C90000000000000001D00000000000000000027
:101CA0000000000000000000000000000000000034
:101CB000005B0000000000000000000000000000C9
:101CC000005F0000000000000000000000000000B5
:101CD0005300585200000050515700595600000060
:101CE0000055000D547E901D04E55893B500150570
:101CF00058E5589370117A0F121D10742D121D3073
:101D00008002D27A755800221477E1F014F077003F
:101D100090E850E0F875A0ECEA7C02B42D027C015A
:101D2000F208B8C0027800D2E7DCF5E8F0D227224A
:101D3000C0E090E850E0F875A0ECD0E0F208B8C040
:101D4000027800E8F0D22722E5592410955A540F62
:101D5000F8E55FC4540FB4040AB80200403F121DF6
:101D60009E8038400CB805004033121DD9402E80AB
:101D70002A204B1F303908E57954F06005800A307D
:101D80004D07B8040040168005B80300400F128DBF
:101D9000C78008B803004005121E42D27322A85A19
:101DA000E60853004F885A75F008A2E7B392F0A2F4
:101DB000E692E7F404A2E792F590E82FF0A85AE63D
:101DC0000853004F885AA2E692E7A2E792F490E8FF
:101DD0002EF090E82DE5F0F02275F008A85AE630D4
:101DE000E74EF4A2E292F0A2E192F2A2E092F108B0
:101DF00053004FE6FE080853004F2690E82EF0EE01
:101E00006630E701B392F41853000F430040E6FE3A
:101E1000080853004F2690E82FF0EE6630E701B334
:101E200092F50853004F885A90E82DE5F0F0C32250
:101E30000853004FC3E559986004E630E7F2885A2A
:101E4000D32275F000A85AE630E6530853004FA29B
:101E5000E592F0A2E492F1A2E192F4A2E392F5A25B
:101E6000E092F2A2E292F3E60853004FA2F292E669
:101E7000C392F2A2F492E790E82EF0E60853004FE6
:101E8000885AA2F392E643F008A2F592E7F404A27E
:101E9000E792F590E82FF090E82DE5F0F022085356
:101EA000004FC3E559986004E630E6F2885AD32221
:101EB000128EE9128A51B4FF058550518006303BDD
:101EC00003D3803D7F3CDFFEC266C2B4D2B2A2D053
:101ED000B37C097E0A7F0030B210DFFBDEF9D2B49A
:101EE000D26680DD121F4C2066171392B4121F5663
:101EF000DCF2121F4CD2B4121F56121F4C121F5686
:101F0000C3D2B4128A2622128EFD128A51303A0AA6
:101F1000C23A855A5980F3D3802C7F3CDFFEC267DA
:101F2000C2B5D2B3A2D0B37C09121F6020671713C9
:101F300092B5121F6EDCF2121F60D2B5121F6E1224
:101F40001F60121F6EC3D2B5128A26227FFF30B2E5
:101F500004DFFBD266227FFF20B204DFFBD26622C1
:0E1F60007FFF780830B306DFFBD8F9D2672286
:101F6E007FFF20B304DFFBD2672278007908E550AB
:101F7E00B55106D8F9D9F7D322A851E6128EE40846
:101F8E0053006F8851C322E4F8FE7902E559B55A21
:101F9E0008D8F9DEF7D9F5D322A85AE6128EF8083A
:101FAE0053004F885AC322E55F5407B40400400122
:101FBE002274FF121EB03066012212113740FA7AD7
:101FCE00017C00121F785004DCF9DAF7121FE2D2FE
:101FDE005CD25D2274F3121EB012113790E863E0EA
:101FEE00121EB012113722C225C24D85595A74FFE6
:101FFE00121F0730670122121F9540687C03121FC3
:10200E009564AA6002DCF7121F95902032E493606B
:10201E001774F3121F07121F95E493A3121F0712D2
:10202E001F9580E9C864500074F2121F07121F95A5
:10203E00121F95C24DB45503D239226002D24D748F
:10204E00E8121F07121F957403121F07121F9574B3
:10205E00E6121F07121F9512207374F4121F071237
:10206E001F95D2252274F3121F07206715121F9594
:10207E007428A8795300F0B850027414121F071276
:10208E001F9522121A3C474F4F440D0A0022121A76
:10209E003C4241440D0A0022121A3C0D0A002275E0
:1020AE00A0E87959E4F319F37C10C3ED33FDEA335C
:1020BE00FA75F002A801430001E235E0D4F218D51A
:1020CE00F0F7DCE675F003A801D375A0E8E230F076
:1020DE0003088001C4540F500D700A20F20330F132
:1020EE000574208003C34430302104F0A3800E30E9
:1020FE005608101E08122D0B8003128552D5F0CAF9
:10210E00302102E4F022301736C217547FF890E8DF
:10211E005CE0540FF94400F5827583EAE8F0E9B506
:10212E0076048879D25DB90400400D7440491222BC
:10213E0008E0122208020D8DE81280B7020D8D30D4
:10214E00E60990E85CF0D217020D8DB4160AD23F64
:10215E0090E867E4F0020D8DB4010B303F031218C6
:10216E00FCD21D020C7CB40C081218C9C21D020D43
:10217E008DB4020812189FC21D020D8DB4150302F4
:10218E0013FAB431061213C4020D8DB43007D248BF
:10219E00C21D020C7CB408087490121EB0020D8D84
:1021AE00A2E792F0C2E7B419004013B43000500E0B
:1021BE00A2F092E7F557755600D27A020D8D020DF8
:1021CE008D301D10540FF576C271C270C21D1217DC
:1021DE0080020D8D304811C248D26DB40400500BF0
:1021EE009092A593457DF57D020D8DC0E074301261
:1021FE002208D0E0122208020D8D200209F82023B9
:10220E0006B4EF03D22322306403FF8016B401021A
:10221E00800CB430028007F85300F0B84004D2644A
:10222E00FE22FE122252E4122289EEA22392E7121D
:10223E008EDA122289306407EF128EDF122289C2E3
:10224E0023C264221222675009B48002D322B481C1
:10225E0002D322F8120B9580EBC310681DC000C08C
:10226E0001780079141222A74006D8F9D9F7740420
:10227E00D001D00030010312855222C0E075A0F4C7
:10228E007819E230E2FCD0E0781BF22275A0F478E7
:10229E0019E230E0FC781BE22290F419E020E00312
:1022AE00C3E42290F41BE0D322FF09FF05030102D1
:1022BE000CFF0A080604462FFFFF4C48FF4A7131F7
:1022CE00FFFFFF7A73617732FFFF63786465343303
:0E22DE00FFFF447666747235FFFF6E6268671C
:1022EC007936FFFFFF6D6A753738FFFF416B696FF9
:1022FC003039FFFF42436C3F703AFFFFFF40FF3C19
:10230C003BFFFF7C49473DFF3EFFFFFF1CFFFFFFEC
:10231C00FF45FFFF11FF1417FFFFFF10601215168A
:10232C00182E7B0B5E135D5C190EFFFFFFFF077D04
:10233C00FFFFFFFFFFFFFF012EFFFFFFFF462F02F6
:10234C00FF4A481C7C713103FF4C7A73617732046D
:10235C00FF63786465343305FF4476667472350622
:10236C00FF6E626867793607FF4D6D6A75373808FE
:10237C00FF416B696F303909FF42436C3F703A0A79
:10238C00FFFF40203C3B0B0D4B49473D3EFF0C0EE5
:10239C0057580F5651534550FF1159141755525455
:1023AC001060121516187B5BFF5F13FF5E195CFF44
:1023BC001B1E2DFF5DFFFFFFFFFFFF4E4F1D6173C7
:1023CC00646668677A7863761C6271776572797473
:1023DC003132333436353B39373A38303D6F753C12
:1023EC006970476C6A406B3F3E41436E6D42464498
:1023FC002F45FF2E4A4F481A4C58595756FFFF602D
:10240C00FF5CFF5EFF7BFFFFFF5B5FFF5DFFFF99E4
:10241C001011121314151617FF1819FFFFFF0506DC
:10242C0007030809FF0BFF0DFF0EFF0AFF0CFF0F40
:10243C00505254510453025501494D4BFF1FFF9EFE
:10244C009C9F9D01020A030B040C054D06A907086D
:10245C00094C560F0D0E58A0A157592E313233345A
:10246C003536373839303A3B2F45509B5B5C1FA2D1
:10247C0060A3524671776572747975696F703C3DD3
:10248C00514B1718195DA4A553FF4A617364666715
:10249C00686A6B6C3F403E475F14151610A654A734
:1024AC007B487A786376626E6D41424349AE111275
:1024BC0013AAABAC9A7C4E444F551C5EFF2D44B115
:1024CC00C0B3B4B5B740B9B0B8BB413A42433031F0
:1024DC003233343536373839BF3FC13BC2C3B2E132
:1024EC00E2E3E4E5E6E7E8E9EAEBECEDEEEFF0F148
:1024FC00F2F3F4F5F6F7F8F9FA3C3E3DB6BA2F6173
:10250C0062636465666768696A6B6C6D6E6F707127
:10251C0072737475767778797ABCBEBDAF1B6030F8
:10252C003132333435363738392D3D5B5D5C3B27E2
:10253C002C2E2F2008090D1B7E2921402324255EDB
:10254C00262A285F2B7B7D7C3A223C3E3F200809C3
:10255C000DB576048B79D25D7583EA4400F582E083
:10256C00B503028004D254EBF0EEF912181CF920DA
:10257C00F71F20F60DE9C45403F9EB1280B7D26DA6
:10258C008041E9C4540F4440122208EB1222088007
:10259C0032E9C45403F8E9540F4440F94303803042
:1025AC00F60F74EF122208E9122208EB12220880AF
:1025BC001274EF1225D6E91225D674EF1225D6EB3C
:1025CC001225D6204A03123DED22C0E0E812847B8E
:1025DC00D0E0C023C2191284A4D02322121A3C0DBD
:1025EC000A00121A3C50726F6772616D2072657628
:1025FC006973696F6E202D2D2D2D20553534440DAA
:10260C000A0022733534642D0090F0007C07786644
:10261C0075F0011280795382F8E5822408F582BCAA
:10262C00040390F400DCEC90F4187888D2F112805A
:10263C007953A8FA121A3C446961676E6F73746916
:10264C0063206D6F64650D0A00903C94122D06E5B5
:0F265C007F0404FC7483122D1C902B09122D2374
:10266B00D20D5389F0438901D28C903C7E122D06FA
:10267B00902B23122D06200D0A7420122289902BE9
:10268B001F80087410122289902B1B122D06E57FD8
:10269B0004B40203E480050303145403F54875499D
:1026AB0000754A007549007590FCD2EC200D05129F
:1026BB0027A88003122710C2EC12291EE549654892
:1026CB0005496014743045491222897C0679401201
:1026DB00229AF709DCF980E1054AE54AB4640375EF
:1026EB004A0074C0122D1C7A00AD4AD21ED256126B
:1026FB0020ADC2560547E547B46408D20C90F800EC
:10270B007408F0809FD202B2027B03754640200210
:10271B0008122A781229108003122A867C047AFB6D
:10272B0080097546407C087AFE0546200203630249
:10273B00FFEABB0406F5C0E5C0800E500844C3F5A4
:10274B00B0E5B08004F5C8E5C86A8A0030020363BF
:10275B0000FF55006004A84646F6E5D8540F60020A
:10276B004243E590543C643C600242447E0475A0B5
:10277B00F07819122901E824F8F8DEF775A0F4783F
:10278B0011122901EA23FA122A2ADCA50B122A9F1D
:10279B001228F0BB068F30020122022712C202124E
:1027AB002A861228F07C047AFB7B03E41229108022
:1027BB00067C087AFE79FCEABB0408F5C0E5C0A8E4
:1027CB00C8801B5013F5B0E5B044C37F001229B786
:1027DB00BF0101F442408022F5C8A8C8E5C07F00C4
:1027EB00491229B7C8491229B7C8BF0106F449C80D
:1027FB00F449C8694241E8694242EA23FAEC30E005
:10280B0007E92323F9122A2ADCAD0BBB06A375C0FB
:10281B000075C800E5D8F4540F6002F5437C0490B2
:10282B00F01B785AE8F023F8E58224F8F582DCF403
:10283B00C2EE90F403E8F0122A951228F07C04788B
:10284B005A90F019E030E00F05820582E0158215F1
:10285B0082B50003C38001D3E54533F545E58224FA
:10286B00F8F582E823F8DCDCE545C333F54590F455
:10287B0011E030E00905820582E065006003434505
:10288B0001D2EEE590543C643CF544A202920ED288
:10289B0002D2EE122A9FE590F4543C643C4244125F
:1028AB0028F090F411E020E70BC2EE122A95E030ED
:1028BB00E7028003434402C202122A861228F0C2A6
:1028CB00B2122A95A20E9202783A122B4090F40182
:1028DB00E030E00A05820582E0B43A02800343430C
:1028EB00101228F022E5905403B40307C2EC759044
:1028FB00FC8002059022E254F1B40100B3E545726D
:10290B00E433F54522E4F540F541F542F544F54352
:10291B00F54522E5415542FD90294A7C045403B408
:10292B000313E493A3FE7F58122A05D20FE49352AC
:10293B004152428001A3A3ED0303FDDCE0800802BA
:10294B00FC01F303CF043F902AE17C14E540030321
:10295B00540FB40F0D7E007F58D20F902AE97C11D3
:10296B008013BC1004E5418005BC0802E54213FD51
:10297B00500D1229C3122A05122A1AD20F8002A354
:10298B00A3EDDCDE300F05122A1AC20FE5436006F9
:10299B001229CC122A1AE5446007031229F0122AD5
:1029AB001AE54560061229F4122A1A2275F008332B
:1029BB0040010FD5F0F93322E493A3FEE493A3FF78
:1029CB0022FD30E4077E007F53122A05ED7F42F58E
:0E29DB00F0A2F092E1A2F192E0A2F292E3A249
:1029E900F392E27E0180087F4480027F507E0013CB
:1029F9005005FD122A05ED0EBE05F422E5496006D3
:102A0900BE000122232324C32E122D1CEF122D0BED
:102A190022D20F79C0E4D9FEC9122A2AC9D5E0F613
:102A290022122A5C4004C2068016200613D2061020
:102A39000C0F754700B40702B20D75810702266DA8
:102A490022C083C08290F800740CF0D082D08375C4
:102A5900470022C006C002C001C000C083C0821264
:102A690030A7D082D083D000D001D002D006227501
:102A7900B0C3E4F5C0F5C8D2EE122A9F2275B0FFA3
:102A890074FFF5C0F5C8C2EE122A9F2274127900AC
:102A9900D9FED5E0FB227C0875A0F07802BC0407BA
:102AA90075A0F47802800ABC03028025BC0102806B
:102AB900207402F2200204747080027460F274457A
:102AC900F2122A9518E230E0070808E2181880F592
:102AD90008E82408F8DCC62200370039003800412C
:102AE90002410239014101390341033904410439E1
:102AF90002380237013801370338033704380437FD
:102B0900433132333435363738393031323334356D
:102B19003600804F5000804C4200C02030004C4F9E
:102B29004F50004F50454E000D0A0020504153535D
:102B390000204641494C00C3122B527C08E813126D
:102B49002B52DCFAD3122B5222CA858AF020F7FACB
:102B5900858AF030F7FAB392B2858AF020F7FA85C0
:102B69008AF030F7FA858AF020F7FA858AF030F78B
:102B7900FACA22E4936006A312855280F622E54937
:102B8900600B902C4D7C04232304FD8019902B2C81
:102B9900200D03902B27122B7C902B31122B7C902C
:102BA9002C317C057D00E57FB401021C1CC083C06B
:102BB90082C001C004C0057A00D22190E810122019
:102BC900ADC22190E811122B7CD005D004D001D0E0
:102BD90082D0830D7907C3E493A3F8E493A35660E5
:102BE90024400FC083C082902B3A122B7CD082D014
:102BF90083D37420128552E493A3128552E493A3DC
:102C09001285528002A3A3D9CE400CC083C0829002
:102C19002B34122B7C8004C083C082902B31122B61
:102C29007CD082D083DC8622400430374010303893
:102C390040083039402031304402313345013235C2
:102C49004310513142083037420430384108303995
:102C590041043130430231314404313345023235C4
:102C690042013037420230384101303941023130B6
:102C7900430131314408313345043235422030377C
:102C89004210303841203039411031304308313158
:102C990044103133450832354280303742403038AC
:102CA900418030394140313043043131442031339E
:102CB9004510323590F8007430F07406F0740CF059
:102CC9002290F800740DF02290F800740CF022752F
:102CD900A0F87900F30975A0F87901E493A36008D5
:102CE900B45C02748CF380F322207710903CD620D8
:102CF9001B03903CEC122D06A21B921C22E493A309
:102D090080CD75A0F87901645C6004645C8002740C
:102D19008CF32275A0F87900F32275A0F87901E403
:102D290093B45C02748CF3A3DCF5227480122D1C1D
:102D3900E576122D577420122D0B7A00AD760DBD54
:102D490000047A017D00D2561220ADC25622120A21
:0E2D59007D7C10122D232290F40F7403F09055
:102D6700F41FF022903CAA122D0622903CC0122D8F
:102D77000622C0E07493122D1CD0E0122D0B229076
:102D87003C68122D06122DCB22903C10122D0622E4
:102D9700903C3C122D06122DCB2290314812329ACC
:102DA700D21690E85F7479F090E85E1230491231DC
:102DB700F622903C52122D06903C7E122D0674C0CE
:102DC700122D1C22903C26122D06122DDD1230A743
:102DD70050FBB407F8221230A740FB123DE4223023
:102DE7005708C25720390312337822E5536002D3BC
:102DF70022307A10AE56BE2E0EC210C27CC2507C54
:102E07002D122F41022EDE201042BE79217C221284
:102E17002F41C250D21090E8377401F090E838E0A3
:102E2700123DB17C107420F0A3DCFC022EDEBE6ED6
:102E3700D390E838E004B5770280034001E4F07CE2
:102E47002D122F41122F02C27A022EE27445A87961
:102E5700B855027451B5061390E837E0B401028003
:102E67007614F0123DB17420F0D322BE4718123DFC
:102E7700CEC21090E838E0B57603122D3490E837CB
:102E8700E0240AFC80BBBE4804D250D322BEC8044B
:102E9700C250D322BE8000503CBE2E004039BE48EF
:102EA70000500E903E73305003903E8DEE93FE809F
:102EB70011BE7B005021BE6100401CEE3050032440
:102EC700E0FE90E837E06411600D123DB1EEF0903E
:102ED700E837E004F0D322C27AC322E4F52CF57A6E
:102EE700C25EC253D322D27C90E838E576F0C25056
:102EF7007A48121D10122F02022EE290E838E0FFE6
:102F0700903D64122F6BD221EF2401FDE43400FAC7
:102F170090E83B1220ADE4F090E83B122F6BC22102
:102F2700903D69122F6BEF120A7D7C10122F7BEFF9
:102F3700120A8C903D6D122F6B2290E850E0F875C5
:102F4700A0EC7445AB79BB55027451F2D2E708B8CF
:102F5700C0027800F2C2E708B8C0027800DCECE8EB
:102F6700F0D22722202104E4938001E06005122F8C
:102F77008980F122202104E4938001E0122F89DC6B
:102F8700F322C083C082903E2293FA53027F20E748
:102F97000C305013C25074C8121D30800A205007DD
:102FA700D2507448121D30C004121D10D004D082B4
:102FB700D083A322903D9B122D0622903D85122D92
:102FC70006903C94122D0622201169201A41203EBA
:102FD70002801090E853E0B41E00400512318C8047
:102FE7000204F0201A2920191330180A123E20A2D1
:102FF700E7B3921B8006123E2EB3921B201C0530AE
:103007001B0D8003201B08303902D25C122CF212F0
:1030170030629257501E90E853E4F0D27990E85FFF
:103027007479F090E85E30221990F800740CF0C2C1
:1030370057C2222290E85DE014F0701EA3E014F05E
:1030470070187404F015827484F090E85FE014F04F
:10305700700890F8007408F0D222221230A74008B6
:10306700C20690E856E4F0229030FA9360F214FE1C
:103077003006028004D3D20622BE0B02800DBE0C9E
:10308700028008BE0E028003BE0F1390E856E004CC
:1030970030E30A2408B4280050DBF080D8F0C322BC
:1030A70075A0F47583F4780D791D75820E7A011277
:1030B70030E7B40F2975820E7A021230E72410B474
:1030C7001F1C75821E7A011230E72420B42F0F755A
:0E30D700821E7A021230E72430B43F02C32278
:1030E500D322EAF0E25403FEE35403232342060508
:1030F50082EAF0EE22000000000000000E00000051
:1031050008000502000000000000000001000000AA
:103115000900060300000000000000000F00000089
:103125000A00070400000000000000001000000075
:103135000D000C0B00201A03122D3422201A031245
:103145002CF222BE0B0BD270D215C26FC2380231DF
:10315500EFBE0C0BD271D215C26FC2380231EFBE71
:103165000A2290E835E4F0123354903D02122D0600
:10317500122CD1D21AC26FC271C2709032A912320A
:103185009A0231EFBE0D15C23EA81F123205403B13
:10319500122CD17491122D1C122D4322BE0A00400F
:1031A50006203E03023247D23EC2381236EC122CBC
:1031B500CAE51FB43D09E577B46300500D800C5096
:1031C5000AE577B409005002800122C23E12322C72
:1031D5004007B5770280074005123195800CF576DA
:1031E500C270C271C238D26FD2151231F6122CD10B
:1031F50022E490E853F0A3F0A3F0751F3BC23E22F2
:10320500B83B02C3227E0090E83BE0CE75F00AA4ED
:103215002E500205F0FEA318B83BEF90E854F0FDE0
:10322500A3E5F0FAF0D32290E855E0F5F0B40200FA
:10323500500E90E854E020F005600514C32260FBB1
:10324500D322C23890E854E576F090325512329A7E
:1032550090E854E0BE0D0DD26FD215F57690314849
:1032650012329A22BE0E0814B4FF10E577800CBE08
:103275000F1904B5770280034001E4F0AF76F576C7
:1032850074C0122D1C122D398F7622122CF290311A
:103295004812329A22C083C08290E85AD0E0F0A347
:1032A500D0E0F02290E835E0F8BE0B0704B40E0C30
:1032B500E48009BE0C2614B4FF02740DA95F530106
:1032C50007B40D05B905E28010B404028008B40CFA
:1032D500028003B40B03B902D0F08073BE0A581004
:1032E5005415C21A90314812329A1231F6122D3401
:1032F500122CF2122CD122903D18122D06903D2E43
:10330500122D0690331412329A90E835E4F022BE5D
:103315000B028003BE0C1290E835E0F4F0903D44BA
:103325006003903D49122D0622BE0DFC90E835E064
:1033350070B012140080ABBE0DBCE823F89039566E
:1033450093F9A3E893F582898312329A0233789030
:10335500E835E0F875F014A42425F582E5F0343A53
:10336500F5837480122D1C7C14122D2312338312C5
:10337500338C2290E85AE0C0E0A3E0C0E022903907
:10338500DAE893122D1C2290E835E0FC9039902361
:103395000493C0E0EC2393C0E022903C7E122D06FE
:1033A500903B3D122D0690E835E0F89039AB7C0056
:1033B500E4A39370030C80F8ECB500F4122CDF74D1
:1033C50029122D0B74D3122D1C122CCA1231F69012
:1033D50036EC12329A22903C7E122D06903B491211
:1033E5002D0674C9122D1C12338C90374C12329A4B
:1033F50022903B54122D06903B7D122D06E5761248
:10340500354A74C4122D1CE576122D57E576120A3D
:103415008C7490122D1C122CCA90E837E4F090E8B9
:1034250036E4F090E838E576F090343512329A2299
:1034350090E837E0FFBE0F080FBF110D7F00800930
:10344500BE0E221FBFFF027F1090E837EFF0700914
:0E3455007490122D1C740D800724C3122D1CC0
:10346300740E90F800F022EF7036BE0B0A1234D3BC
:1034730004B50010E4800DBE0C5E1234D314B4FF07
:1034830003E50014F090E838E0FF12354A74C412E3
:103493002D1CEF122D577490122D1CEF120A8C2243
:1034A300BE0B0B123DB104B47E107420800CBE0C15
:1034B30027123DB114B41F02747DF0F8122CD1E829
:1034C300122D0BEF24C3122D1C740E90F800F02262
:1034D300A8770890E838E022BE0A13122CD1748032
:1034E300122D1C7C14903A9D122D23023774BE0DAD
:1034F3001990E837E06013123DCE90E837E4F0749A
:1035030090122D1C740D90F800F022903B54122D54
:1035130006903B67122D06E57612354A120FC2124A
:103523003557120FC21235707490122D1C122CCA0B
:1035330090E837E4F090E836E4F090E838E576F088
:1035430090359E12329A22C0E07491122D1CD0E065
:103553001237AE22780E540F14F5F074C3122D1CDB
:1035630012369F1236CA90E839E5F0F022F8540F6C
:10357300B40400400824FDF5F07803800CE8C4543B
:103583000F9037DE93F5F0780474CA122D1C1236AF
:103593009F1236CA90E83AE5F0F02290E837E0FF50
:1035A300BE0F080FBF030D7F008009BE0E381FBF7B
:1035B300FF027F02BF020990E839E0B4030050E044
:1035C30090E837EFF0122CD1903E03E493600B1296
:1035D3002D1C741D122D0BA380F1903E03EF93124B
:1035E3002D1C122CCA22BE0B0A123E0704B5001072
:1035F300E4800DBE0C4B123E0714B4FF03E5001428
:10360300A982B9380AC0E012366CD0E090E838F0ED
:1036130090E838E012354A90E837E0700E90E838C9
:10362300E07583EA4400F582E0800312367AC0E055
:10363300123557D0E012357090E837E0FF1235DDD0
:1036430022BE0A1C90E837E0700312366C122CD1AC
:103653007480122D1C7C14903A89122D2302377426
:10366300BE0DDD90E837E0D25412367AFB90E8388D
:10367300E0FEC24A02255D90E839E090368893B4B3
:1036830044004006220102034455F890E83AE090D2
:1036930038AF9354F0482290E835E0F89039E9E8E0
:1036A3009390E830F09039F8E89390E831F0903A4D
:1036B30007E8230493F9E8239390E833F0A3E9F0B0
:1036C3002290E832E0F5F090E830E0FCC0F0A4D0BE
:1036D300F0F990E830E0FC90E833E0F8A3E029F556
:1036E30082E438F583122D2322A81FBE0A00500F4F
:1036F30075A0E8EEF208B83F131818F208800DBE63
:103703000E028003BE0F3218B83A0108881F749165
:10371300203E0274D1122D1C123205400A903C7FC8
:103723007C03122D238007D2561220ADC256749308
:10373300203E0274D3122D1C22BE0A028033BE0D1A
:10374300F7123205403E02394590E831E0F890E83F
:1037530032E0BE0B0704B5000CE48009BE0C0F1465
:10376300B4FF02E814F074C9122D1C1236C4BE0A49
:1037730010903D02122D06122CD19032A912329ACA
:1037830022BE0D1B90E835E0F8B400028002D2544B
:1037930090397493E8230493C0E0E82393C0E022B4
:1037A300E4A23892E0FC023842E5772401FDE434D8
:1037B30000FA02384EE55F540FB402057C0002386C
:1037C30042B404047C018077B405F17C028070E587
:0E37D3005FC454079037DE93FC806400000151
:1037E10003000290E86EE0FD90E86CE0FA53020FEE
:1037F100805B90E904E0FC804890E86AE0FD90E895
:1038010068E0FA53020F804590E863E0F4541FFD2D
:103811007A00D21E803790E863E0F4546003C4FC60
:10382100801F90E930E0FD7A00D21E802090E8668A
:10383100E0FD7A00D21E801590ED00E0FD7A008057
:103841000C12369A90E832ECF01236C422D256129B
:1038510020ADC256C21E2290E832E0A2E0923802A8
:10386100393F12322C40046002F57702393F90E86B
:1038710032E090389593F9540FB40209E55F540F83
:10388100B40202A95F895FC00012063812073CD05A
:103891000002393F12445590E832E09038AF93F579
:1038A1005FF9895FC00012073CD00002393F122244
:1038B100523290E855E090E86CF0A3F090E854E0C3
:1038C10090E86EF0A3F0807690E832E090E904F0A1
:1038D100806C90E855E090E868F0A3F090E854E03F
:1038E10090E86AF0A3F0805690E854E0F4541FFC8D
:1038F10090E863E054604CF0804490E832E0F45486
:103901000323C4FC90E863E0541F4CF0803090E83E
:1039110054E090E930F0802690E854E090E8665455
:103921000FF0801A90E854E090ED00F0FEC000E442
:103931001222897403122289EE122289D0001233D5
:103941008312338C122CD1903D02122D069032A994
:1039510012329A222233DB339F33DB33DB33DB3505
:103961000E33F6339F339F339F339F339F33DB33C4
:103971009F339F385838B338C9386F38983955391B
:10398100553863390F391938D338E938FB392537B8
:10399100A337E437F337B837D23955395537AC380F
:1039A10023382E37FA38093817383900312D39398B
:1039B10039000000000000322D32353600312D3142
:1039C1003600312D313600312D39393900322D3360
:1039D100300000302D323535008B8C8F8A87D4D45E
:1039E1008F919191928A91D40300030A0A000000F9
:1039F10000000000070003020002030400000000B1
:103A01000000000400053BDF00003BD93B933BB1C4
:103A110000000000000000000000000000003BE585
:103A210000003C015363616E206D6F64651D2020B1
:103A310020202020202020205363616E2074696D96
:103A4100651D20202020202020202020506F776518
:103A510072206F6E207363616E1D20202020202054
:103A61004B6579626F6172641D2020202020202027
:103A7100202020204D6F7573651D202020202020DF
:103A81002020202020202020435055206B65796282
:103A91006F6172642F6D6F757365202043505520DF
:103AA1006E616D65732020202020202020202020A1
:103AB1004D6178696D756D20706F7274731D202072
:103AC10020202020457870616E73696F6E207769C0
:103AD1006474681D20202020457870616E73696FC1
:103AE1006E20756E6974731D2020202056696465EF
:103AF1006F20626C616E6B2074696D651D202020E2
:103B01004B422072617465206B6579732F73656315
:103B11001D2020204B422064656C61791D202020EE
:103B2100202020202020202053756E206B62206CE5
:103B3100616E67756167651D20202020C04E657725
:103B41002076616C75652800C043686F6F73659E50
:0E3B51009F20008043686F6F7365209E9F7FEA
:103B5F007E20204350551D00C04B421D20202020A9
:103B6F004D531D2020202020202020202000C04E3B
:103B7F00616D652020202020202020202020202063
:103B8F0020202000504320202020202020204D6185
:103B9F00632020202020202053756E2020202020FD
:103BAF00202050532F322020202020205365724D8B
:103BBF006963736F667453657250436D6F75736588
:103BCF00536572204F74686572204E6F205965736C
:103BDF004F66664F6E20536C6F772020204D6564C3
:103BEF0069756D204661737420202046617374657A
:103BFF0073745043315043325043334D61635375A7
:103C0F006E80526573657420737563636573736635
:103C1F00756C2020202000C048697420656E746583
:103C2F007220746F2070726F6365656400805265D7
:103C3F00736574206661696C6564202020202020E4
:103C4F0020200080436F6E66696775726174696FBB
:103C5F006E207265736574200080436F6E666967AE
:103C6F0075726174696F6E2062616420202000C0DC
:103C7F002020202020202020202020202020202035
:103C8F0020202020008020202020202020202020E5
:103C9F002020202020202020202000C050726F677D
:103CAF0072616D20636F727275707465642020206D
:103CBF0000C0536C617665206C696E6B2062616425
:103CCF0020202020202000C05374617475731D20A4
:103CDF006E6F726D616C20202020202000C0537405
:103CEF00617475731D206E6F2063707520706F7710
:103CFF00657200C0456E746572A573656C656374FB
:103D0F00209E9FA56974656D008053617665206361
:103D1F006F6E66696775726174696F6E202000C07F
:103D2F00456E7465722063686F6963659E9F205945
:103D3F006573202000CF59657300CF4E6F20008030
:103D4F005363616E206D6F6465202020202020203A
:103D5F0020202020004E616D6500203D2000204373
:103D6F0068616E676520592F4E2F4553433F2000E2
:103D7F004F6E204F6666C05374617475731D206E4D
:103D8F006F742073656C656374656400C0537461F0
:103D9F007475731D20766964656F206F66662020C9
:103DAF00200090E838E05403C4F890E837E014544A
:103DBF000F42007583EB7400543F48F582E02212E6
:103DCF00094690E838E0120A7D5382C075A0EB795E
:103DDF00001215492278007900D9FED8FC2290E80C
:103DEF0037E4F0FF123DF722903E03EF93122D1CA4
:103DFF00122CCA2290C2C900BF0107780590E8397A
:103E0F00E022780490E83A5006A8770890E838E066
:103E1F0022E575C4540F4410F5827583E9E022C082
:103E2F00E0740925748355D8D36001C3D0E0220212
:103E3F0001080444B1C0B3B4B5B740B9B0B8BB4181
:103E4F003A424330313233343536373839BF3FC1D8
:103E5F003BC2C3B2E1E2E3E4E5E6E7E8E9EAEBEC13
:103E6F00EDEEEFF0F1F2F3F4F5F6F7F8F9FA3C3E78
:103E7F003DB6BA2F6162636465666768696A6B6C89
:103E8F006D6E6F707172737475767778797ABCBE58
:103E9F00BDAF1B60303132333435363738392D3DB5
:103EAF005B5D5C3B272C2E2F2008090D1B7E2921E3
:103EBF00402324255E262A285F2B7B7D7C3A223CDB
:0E3ECF003E3F2008090D2030362F31302F39AC
:103EDD003820436F707972696768742031393930D1
:103EED002D3139393820526F736520456C656374F7
:103EFD00726F6E69637320C2A91290C175F02C1296
:103F0D003FE512400612402B20083F123FB2403AC7
:103F1D00D20ED279A950A7060953016FA707B7FF93
:103F2D0002800EB7B607E506B4B602800409530148
:103F3D006F89503001147420128552744B128552C2
:103F4D00E506128534E5071285341290CE128A26C5
:103F5D00D2A922128A51C2A91290C175F03C123F0A
:103F6D00E512400612402B200832123FB2402DD2EE
:103F7D000DD279A959A7060953014FA70709530176
:103F8D004F8959D249300114744D128552E50612EC
:103F9D008534E50712853474201285521290CE12A5
:103FAD008A26D2A92212403B402D7D0812403B406B
:103FBD0026300903C38001D3E50633F506DDED7D1B
:103FCD000812403B4011300903C38001D3E507338C
:103FDD00F507DDED12403B2253B0CB7C9200000083
:103FED00DCFB43B0347C1ADCFEE5F07D0833124077
:103FFD00890000000000DDF52253B0CB7C1FDCFEF4
:10400D0043B0347C0DDCFE20B4028004C208800D68
:10401D007CFF20B406DCFBD2088002C20822C20855
:10402D007C3F30B406DCFBD2088002C208227CFF44
:10403D00DC02801D20B4F97C000C30B4FCC3EC9480
:10404D000E500AC3EC94034008C2098002D209C382
:10405D0022D3227C26DCFE227D10C5F0D3124089AE
:10406D000000000000000033124089BD0904C5F0B6
:10407D008003000000DDF0C312408922C0E053B080
:10408D00CB7C0D500280027C1BDCFE43B0347C13D4
:10409D00500280027C05DCFED0E0227C127DFFDD2B
:1040AD00FEDCFA22128A51C2A91290C175F02B12B0
:1040BD003FE512400612406075F06275E003124054
:1040CD00651290CE128A26D2A9224300F830E0055F
:1040DD005300FB800343000430E1055300FE8003D1
:1040ED0043000130E2055300FD8003430002E5006B
:1040FD00221240D785E0827583FF128A51C2A91220
:10410D0090C175F02A123FE512400612406085827B
:10411D00E08583F0124065C20C1290CED2A9222206
:10412D0002974C32FFFFFFFFFFFFFF758C10D26B24
:10413D00327583F011607583F411601286997900E0
:10414D007583E8E92480F582E07583EAF582E01253
:10415D0080B709B904EA90F400786675F000E55F60
:10416D005407117990F410117990F408787775F05F
:10417D0003117990F41A7415F07582187403F022F6
:10418D0075821274C0F075820FE075821FE0758222
:10419D00047470F0758214F022438202741AF0F0E8
:1041AD005382F8438200741330F2027407A2F09226
:1041BD00E0F07407F05382F8438201E8F05382F87F
:1041CD00438202748020F1027490F074A020F102F9
:1041DD0074B0F07405F022C4540F75F0007866B415
:1041ED000500401AB4050575F0018012B406077577
:1041FD00F00578668008B407F375F001789975833A
:10420D00F0E9C403F58212807922E590543C537D88
:10421D00C3427D227583F030E3037583F4C4032418
:10422D0001F582E030E20D5382F8438203E8F0128B
:10423D008F11C322D3755D0022E8B57800401B9025
:10424D0092A193FE55906004EE427D22EE557D6065
:10425D0009E8784D11F4EEF4527D22F9E574917B65
:10426D0074EF91A4E574917BE991A42279387B30A8
:10427D00D255E95403C074F574B120D07450028046
:10428D0053E578601BE95403F8B57800500280348B
:10429D0090E930E08578F0A428C39578F582800701
:1042AD00E954032400F5827583EAE05407B4070549
:1042BD00128356801FB40402801A40045195801455
:1042CD00E0C45407D1CA430104D1CA5301FBE954D8
:1042DD0003F83119090B309803128A8CB93C93C23B
:1042ED005522128E80128520204E49404720020310
:1042FD0020182BE5795407B40707E5741280F48074
:10430D002AB4041175F0FF128F4C50280554E55452
:10431D00B40A2A801F4007E57412858F8016E57454
:10432D0012847BE890E885F01284B550070554E5BA
:10433D0054B4A00975540005551553C322D3221248
:10434D008520204E685002806420020320183DE530
:10435D0079C45407B4041888F009E3F8128F635038
:10436D000A055DE55DB40A4C755D00755C00224083
:10437D0011B40707E5741285FF8032E5741280F4DD
:10438D008022B40207E5741280F48018E5749092CF
:10439D00A593557D6017E574D2E212847BE81284F3
:1043AD00B5500A225007055DE55DB4A007755D00A7
:1043BD00055E155C22E754036002801AE95403126E
:1043CD0083A0400122B71005770051B822B40139FE
:1043DD0077037E0051B880737583E9E95403F8447F
:1043ED0010F582EEA2E292F0A2E092F1A2E392F237
:1043FD00A2E192F3E5F0540FF0E576200205E575A4
:10440D00C4540FB50044D25C22B40E067710128945
:10441D007922B40F0477068032B402028010B403FF
:10442D0002800BB40A028006B40B02800122E9540B
:10443D0003F8E576200205E575C4540FB5000B9021
:10444D00E8402582F582EEF0D27522E790974393EE
:10445D00B4040E90ED00E0A2E77404500D740380D7
:10446D0009B45A0690ED00E0547FF8E95403128523
:10447D008F171289792290F41112838950117420AB
:10448D00B152746BB152E8B13490F0011283969031
:0E449D00F00112838950117420B1527463B182
:1044AB0052E8B13490F40112839622E020E002C36B
:1044BB0022438203E0F8D322E030E2FC438203E89C
:1044CB00F0227583F0F830E3037583F4C403240101
:1044DB00F582E020E004C3E4800B5382F8438203AF
:1044EB00E0128F16D3FE22A2E2924AC0E0917BD05B
:1044FB00E054039084A093C002FA128A517C08788E
:10450B00009144E5C8304A02E5C05AC36001D3EEBE
:10451B0013FEDCED9144E5C8304A02E5C05A600158
:10452B000C9144E5C8304A02E5C05AC24A6002D237
:10453B004AC39126E572F442C8E573F442C0128A6D
:10454B0026D002ECA2E0EE22C0E0400AE57252C88F
:10455B00E57352C0800AE572F442C8E573F442C0B9
:10456B00D0E07F0180027F04DFFEC0E0E57052C81F
:10457B00E57152C07F0EDFFEE570F442C8E571F4C1
:10458B0042C0D265E570F4600855C88009C0E08070
:10459B00F1E571F455C07002C265D0E022FE2055E2
:1045AB000430190122A2E2C2E290849C937FFF4067
:1045BB0001CFF57103F573CFF57003F57222F7FD9B
:1045CB00DF7F040110407D00C0E0128F2A1284CBE4
:1045DB00D0E05002DDF222205506301903022208EA
:1045EB00BE04005005128EEE8003128F02FFEEA266
:1045FB00E2C2E290851C93400445C8800245C0CFBF
:10460B00BFFF028002D322128A5112846B30651EC7
:10461B00C3128426306517A2D0B37C0913128426EB
:10462B0030650BDCF7D3128426C3128A2622D3FC07
:10463B00E572F442C8E573F442C0ECD380ECF3FCB2
:10464B00CF3FC0E0740925748355D8D36001C3D024
:10465B00E02202010804300111C0E0C4540FB1493B
:10466B00D0E0C0E0540FB149D0E022B40A004002C0
:10467B0024072430300107F5993099FDC299229017
:10468B00E857E0D5E0027406F0B406247938E7B4B5
:10469B00100280045403600FB24020400A7700538D
:1046AB0001F77700430108E52803F52809B940DE37
:1046BB0022C8128F1BC890972993FAC3B1A87C0804
:1046CB00E813B1A8DCFBD3B1A822CA858AF020F786
:1046DB00FA858AF030F7FA400452C88004F442C8D5
:1046EB00F48024C8128F20C8C3B1D57C08E813B15D
:1046FB00D5DCFBD3B1D522CA858AF020F7FA858A9F
:10470B00F030F7FAB392B2858AF020F7FA858AF087
:10471B0030F7FA858AF020F7FA858AF030F7FACA73
:10472B0022C8128F1BC890972993FAC3D11C7C09FE
:10473B00E8A2D0B313D11CDCFBD3D11CC322CA8596
:10474B008AF020F5FA858AF030F5FA4006F442C873
:10475B00F4800252C8858AF020F5FA858AF030F58C
:10476B00FA858AF020F5FA858AF030F5FACA22AC80
:10477B007420020CE57554C07023E575C45403FC1A
:10478B0074382CF82404F9E6B41001225403700F8A
:10479B00E7B4100122B434012254037002D322C3B4
:1047AB0022C320020DE57554C0700EE575C4540389
:1047BB008002E576B50402D322C3227C0075A0E803
:1047CB007880EC20021F12867F401890E930E0F5CC
:1047DB00F0ECB578005003A4800BE578A42CC395BE
:1047EB00788002E576F2080CBC04D722E9540390DA
:1047FB0084A093FAE9A2E2E5C85002E5C0FE5A7024
:10480B0044EE035A603F5012E5C8FE5A7007EE03A0
:0E481B005A70028030E5C05A702BE9540771C4
:10482900C5304A0F20D0045004800A50087433C29E
:104839004A80027422B93C005005128EF38003129B
:104849008F07304A0280030287B2E7B4100AE920D1
:10485900E22CBEFF320287ECE930E2F912874FB44D
:10486900EEF3BEEC030287ECBEFF030287ECAC0655
:10487900028806540390E87C2582F582E02212879B
:104889004FB4F303128988770DE920E24954039064
:10489900E840FC2582F582E0B4ED1FEE7583E98CD2
:1048A90082438210F0D17F502DE07583E98C8243D9
:1048B9008210F0D25C02884E8056B4F019EE70195D
:1048C900ECB5780085768240028C827583EAE054E3
:1048D9000323232416F70289071289675407B404AE
:1048E90000501BEE30020D30E70AA2E45403B392E4
:1048F900E4F0800AE054F05306034EC2E7F0D17F9A
:104909005070EEA2E79207C2E7E0F579D25D8062C6
:1049190090921F7C45B93C0040059092437C65A369
:10492900A3ECB58250B465077CFEE954078012BE3A
:10493900FE19E954037CFAB5740790E885ECF0E5B3
:104949007412847BEC1284B5028907128967B45505
:1049590006EE1282F9801775A0E8E954032440F89D
:10496900E2F87429B8FE005014B8FB00400F740D2A
:10497900770D028907E493B506A5A3E493F7E954F3
:1049890007A2E2C2E290E840500390E87C2582F554
:1049990082EEF0E9540730E271C2E2B57400BEF26A
:1049A90019E95403B578005005774202890712893D
:1049B9006754F07002773A028907D2E2BEE924759A
:1049C9000504F5007C14E812847BE505240F83C0F7
:1049D900041284B5D0045002DCECD505E9804C3CC6
:1049E9000390FA9092A5540393BEF404427D803B50
:1049F900BEF50B2018F82019F5F4527D802DBEFF65
:104A0900EDC0E01289DFD0E080E9BEFF1E7583E9C1
:104A1900E95403F582438210E4F012896754F044A3
:104A290002F0E95403FC12867F925CE7B4340280F9
:104A390004540360558B0006E6FEE7B408005007EE
:104A49009091D5936E7043E9A2E2E5C85002E5C0A2
:104A5900035A7003168033E95403C074F574128540
:104A690020D0744025E9540712847BE79091DD93A7
:104A7900FCE95407B5740590E885ECF0EC1284B5AF
:104A890050031680051776003179227583E8E954B9
:104A9900032480F582E07583EAF582E022E924CBDC
:104AA90083522822FEFDFBF7EFDFBF7FBEC80280DD
:104AB9003CBE64081289CFB4C8318031BE502C1273
:104AC90089CFB46426C3204D01D3C0D0128967D0E1
:104AD900D0540F50024410FEE95403B57800400B3E
:104AE900CEF0CEFC12867F50028E797E001289D4D8
:104AF900EEF0221289D4E02290E878E95403258265
:104B0900F58222C006D31289A67E001289C9D00671
:104B190022201835201932128520204E2C402AE5F2
:104B290079B4440975F0FF78B6128F4C22B4550F49
:104B3900E574780D12858FE574788D12858F22B40E
:104B49007707E57478B31280F42220022530AF2468
:104B5900C0E0203B12E55F64446015E55F64556081
:104B69000FC289D2A8D2B2203A06C28BD2AAD2B336
:104B7900D0E0D2A92220023530AF3430A816202F38
:104B8900FD203B10C2A87CFF20B204DCFBD266C228
:0E4B9900B275250830AA162037FD203A10C24A
:104BA700AA7CFF20B304DCFBD267C2B3752608C218
:104BB700A922200236205E33205930205A2D205852
:104BC7002A203D27205C24205D21203C1E205B1BE2
:104BD700C3E5592410955A540FB40900500DE599AF
:104BE700C298201207B43F0485769922F599309927
:104BF700FDC29910124C205E48B40005D212C220A3
:104C070022B40105D212D22022F890E852E0C8B4AB
:104C17000D1518E577B50000400A8876C270C238CE
:104C2700D26FD215E4F02224D0B40A005013C8C0C2
:104C3700F075F00AA4D0F030D2028005285001E4C4
:104C4700F02220200AA850F60853006F885022A8A7
:104C570059F60853004F8859D24922855600755393
:104C670000E579540FFE300205200705800C301847
:104C7700097E03B4030050027E0275A0E87920BEC6
:104C87000402801FB81A028003B89A17EE14232370
:104C9700FE909265755300EE936007F3090E055376
:104CA70080F522E86007A2E792F0028BCBBE0303F0
:104CB700028C134011E557A2E792F0C2E7B419003E
:104CC70040EEF8028C52E557B4050050E374E0F368
:104CD70009755301E5571423255714F8909285BE9B
:104CE7000103909279E89360070553F3A30980F5D0
:104CF70022BE0133E8547FB40F0C30F002803A90A3
:104D07009291780080DF917A6009A2F092E7F375BB
:104D17005301229092A974E0F309E8547F93A2F01B
:104D270092E7F375530222BE0247E8547FB41F038C
:104D3700301806B40F0E30F0047553002290929885
:104D4700780080A1917A600F75530130F00674F0F6
:104D57000553F309E8F32290932975530274E0F39E
:104D67000930F00974F00553F30953007FE893F312
:104D770022BE0304917A80D0BE040491A28003BEB0
:104D8700051DE5567014B81905BE04AD8003BE05B0
:104D9700A8909714E8C2E79361E4917A61E422222C
:104DA700EE149093A9C0F075F080A424A9F582E5CC
:104DB700F0D0F03493F583E8C2E793B4FF06D0E070
:104DC700D0E081136001F822B81A03D38004B89A9F
:104DD70009C3D1A992E2F0D25C22B87C16D1A9D23C
:104DE7005CB2E2F0D2F078FC30E207C2F0787C7572
:104DF700530122B8FC06D0E0D0E08113B87B06D17E
:104E0700A9B2E18007B80E07D1A9B2E0D25CF022BF
:104E1700D27375A0E87928E579C4540720192B20A7
:104E27001823B40706D138755C0322B40406B127EA
:104E3700755C02224006B151755C0522B40206B1C9
:104E4700F4755C03226003B1AF22B1B32290E82D61
:104E5700E0F5F0A3E0A2F492E6D2E790E829F0901B
:104E6700E82FE0A2F592E7F404A2E792E6A2F0B3F6
:104E770092E790E828F02290E82DE0F875F080F4AA
:104E8700A2E092F2A2E192F0A2E292F1E5F090E8BC
:104E970028F088F0A2F490E82EE090E829B185A2E6
:104EA700F590E82FE090E82AB18522401420E70426
:104EB7007800801B04F853007F7002787F747F802E
:104EC7000EB48000400478008005D2E7F87480F0C3
:104ED700A3A3E8F022740380027404FCF55C90E855
:104EE7002D75A0E87828E0F208A3DCFA22A85A90EA
:104EF700E82D7C03E6F008A353004FDCF7200211EE
:104F0700303908E57954F060088003204D03E480C8
:0E4F170002E608F053004F885A2290E82DE081
:104F250075F040A2E092F5A2E192F4A2E492F1A21A
:104F3500E592F390E82EE0A2E692F0543F90E8293E
:104F4500F090E82FE0A2F392E7F404A2E692F2A231
:104F5500E792F3543F90E82AF090E828E5F0F02234
:104F650090E82DE075F090A2E092F2A2E292F1A213
:104F7500E192F0A2E4B392F4A2E5B392F390E82EA5
:104F8500E07002D2F430E702F40490E829F090E8EA
:104F95002FE07002D2F330E702F40490E82AF09093
:104FA500E828E5F0F0222222E5795407B4040474D8
:104FB5007F80044017743068A2E7C2E7700EE5747D
:104FC500908EA5934004F452C02242C022080220CC
:104FD50080E576200205E575C4540F4410F5827509
:104FE50083E9E022751E748076751E738071751EC7
:104FF50053806C751E6D8067751E2A8062751E2B29
:10500500805D751E798058751E7A8053751E6B807C
:105015004E751E4B8049751E638044751E43803F47
:10502500751E78803A751E588035751E70803075EE
:105035001E50802B751E758026751E718021751E6C
:1050450051801C751E628017751E428012751E7276
:10505500800D751E778008751E6D8003751E6E3078
:105065000111C0E07420128552E51E128552D0E070
:1050750012853422C20DD20E30010CC8128F2FC8F2
:10508500C5F0128F2FC5F012912222D20DC20E301B
:10509500010CC8128F34C8C5F0128F34C5F01291B7
:1050A5002222C20843C83E7C0FDC02804D7DFFE50D
:1050B500C8553C6004DDF880F07C000C0000E5C8B4
:1050C500553C60F7C3EC9467500A20082D1291CC2B
:1050D500D20880D07C000CE5C8553C70F9C3EC942F
:1050E50009500280157D08129096400E300903C3C1
:1050F5008001D3E833F8DDEFC322D322300A16E569
:105105003F52C8E53D52C07C68DCFEE53C42C0E547
:105115003E42C8C20A2200E8B42A06D20BD20C804D
:105125004FC20BE854F3B42009300E3EC20ED20F25
:10513500803AE854F3B43009300D2FC20DD20F80F8
:105145002BE854F3B4220A8EF08FE0C20ED20F8002
:105155001B8017E8B42F0C75F06375E002C20ED200
:105165000F8009E8540FB40B0100C20F7C5FDCFE11
:10517500227D10C5F0D312906D00000000000000E4
:105185003312906DBD0904C5F08003000000DDF009
:10519500C312906D22C0E0E53F52C8E53D52C07C88
:1051A5000B500280027C19DCFEE53C42C0E53E4224
:1051B500C87C13500280027C06DCFED0E0227CFF16
:1051C500DC028023E5C8553C70F67C000CE5C8552B
:1051D5003C60F9C3EC9408500AC3EC94044008C23F
:1051E500098002D209C322D322853C1E853D1D8537
:1051F5003E1C853F1B22851E3C851D3D851C3E852D
:105205001B3F227C26DCFE8015129096C2087CFF8F
:10521500E5C8553C6006DCF8D2088002C2082212B7
:10522500909640257D08129096300903C38001D3DE
:10523500EE33FEDDF17D08129096300903C380013F
:10524500D3EF33FFDDF112909622888285F0831229
:105255008A511290C11291A3128F7A402F12916B2D
:10526500300A028002800B128FD48582E08583F09C
:1052750080E6128FEE200B0E300F118582E08583BC
:10528500F012904980061290DB1290F71290CE1220
:0E5295008A2622200D028003200E2DE854F000
:1052A300B400028021E854F0B42010E8B42E0302C5
:1052B30091A0E8B42A028012200D0BE854F0B43018
:1052C30009200E028004D20A8002C20A22C082C0D0
:1052D30083E5749091C493F53C64FFF53DE57490C8
:1052E30091C893F53E64FFF53FD083D08222040139
:1052F30010400C0330C07C047DC8DDFEDCFA2200C4
:105303000A01000001030100AAFA000000AAFA0042
:1053130083ABFA00FA000000FA00000000FA000074
:1053230001FA000002FA000003FA0000EE00000098
:10533300FE000000BFB0FA00000008FA0000000001
:1053430003FA0000FC00000055FA00FF02F20BED27
:1053530011F311F40DF011F50DF60DF70DF80DF92C
:105363000DFA0DFB0DFC0DFD0DEE25D229EF2FFFE0
:1053730007F60DF50DF40DF311F216E811E70DE63E
:105383000DEA0DE900EC0DF00DEE0DEB34E43D3AC2
:10539300BA000058F0580014F01400000000007721
:1053A300F77F002A0000360000AA0000B6000012B2
:1053B3000000590000F01200F05900E11D45E19D85
:1053C300C500E11477E1F014F07700040810200120
:1053D3000240800000000000000000000000000008
:1053E3003700000000000000000000000000000083
:1053F3005D0000000000000000000000000000004D
:105403000000000000000000000000000000000099
:1054130000000000000000000000000000001D006C
:10542300385B5C5253474F495148504B4D00350050
:1054330000001C000000000000000000000000004D
:105443000000000000000000000000000000000059
:105453000046000000000000000000000000000003
:105463007C000000000000000000000000000000BD
:105473002F000000000000000000000000000000FA
:105483000000000000000000000000000000000019
:1054930000000000000000000000000000001400F5
:1054A300111F2770716C697D7A75726B74004A00E5
:1054B30000005A000000000000000000000000008F
:1054C30000000000000000000000000000000000D9
:1054D300007E00003B3C3D3E3F4041424344575821
:1054E3000046FF524F50514B4C4D474849FFFF5622
:1054F30000FFFF2BFFFFFFFFFFFFFFFFFFFFFFFF8C
:10550300FF01290B02030405060708090A0C0D1AFB
:105513001B2B2728333435390E0F1C2A361D003830
:1055230000000000000000000000000000FF003742
:105533004A4E00531E302E201221222317242526E3
:105543003231181910131F14162F112D152C453A2B
:105553005400FF000506040C030B830A01097807B6
:10556300007EFF7069727A6B73746C757DFF606186
:105573000062625DFFFFFFFFFFFFFFFFFFFFFFFF13
:10558300FF760E45161E26252E363D3E464E5554B5
:105593005B5D4C5241494A29660D5A125914001158
:1055A30000000000000000000000000000FF007C7D
:1055B3007B7900711C322123242B3433433B424B30
:1055C3003A31444D152D1B2C3C2A1D22351A775890
:1055D3008400FF00070F171F272F373F474F565EE3
:1055E300575F627069727A6B73746C757DFF801399
:1055F3008D818153FFFFFFFFFFFFFFFFFFFF80FF51
:1056030082080E45161E26252E363D3E464E55541F
:0E5613005B5C4C5241494A29660D5A125911EE
:105621005819398B8C67646E656F6D6360616AFFB1
:10563100777E847C79711C322123242B3433433BC4
:10564100424B3A31444D152D1B2C3C2A1D22351A53
:105651007614FFFFFF007A78637660616264656D9E
:10566100676F696B7152535455565758595B5C3982
:10567100370A7F7F7F2AFFFFFFFFFFFFFFFFFFFF4B
:10568100FFFFFF35321D1213141517161A1C191BB3
:1056910018211E2A29272B2F2C3133302438383654
:1056A100363A3A37377275737774793E3D3B3C51E0
:1056B1004B434E454C41000B08020E0305042226C4
:1056C10028252E2D1F230C0F011120090D0710066F
:1056D1004739FFFF39000506080A0C0E10111207A1
:1056E100090B1617155E7071725B5C5D444546FFD0
:1056F100FF7C30303058FFFFFFFFFFFFFFFFFFFF50
:10570100FFFF7F1D2A271E1F202122232425262853
:105711002940415856576B6C6D792B3559636E4C46
:1057210043130D787A2C42344A607B141B181CFFFA
:105731002E2F477D5A324D68664F385051523D5396
:1057410054556A693E3F36394E3A3C6737653B648A
:105751006277FFFFFFFF565758595A5B5C5D5E5FEA
:1057610060616263643A393F403E444542434AFFC7
:10577100FFFFFFFFFFFFFFFFFFFFFFFFFFFFFFFF38
:10578100FFFFFF06362D070D0E15161D1E25262EB1
:10579100353037382A312C3334523C083205040273
:1057A100555354FFFF653D666867695049484FFF8F
:1057B1006B6C4B6D51410A231B111012191A2721D1
:1057C10022292B24282F09170B18201C0F141F1313
:1057D1006A03FFFFFF00565758595A6465666768A8
:1057E100717281828392969798999A9B9D9E9FFF51
:1057F100FFFFFFFFFF73747C7D80A0FFFFFFFFFFB2
:10580100FFFFFFBFC9EFC0C5CBD0D6DBE0E5EAF9AA
:10581100F5FAF6F7F2FBE8EDF3D4BCBEBDAEABAFE3
:10582100ADACB2B1FF888C8A8D8E8FAAA9A7A8FFD3
:10583100A2A3A4E89594C2D9CECDCCD2D8DDE6E21C
:10584100E7ECE3DEEBF0C1D1C7D7E1D3C6C8DCC3D7
:10585100A1B0FFFFFFFBFEEFBF51762D0204010354
:10586100191A313348495F61300F7374757F6F00C6
:105871007F04FF005AFE000075B0FF75810775E8CF
:105881000475D8DF7590FCE4787FF6D8FDE590F4D7
:1058910054C02440F57F60FE74FFF5757550607546
:1058A1005160755940755A40757B00757C0090E8D0
:1058B100577406F0D202129BA7B4E6FA129BA7FC1A
:1058C10090ED00129BA7F0A3DCF9E57FC4FE90E9FF
:1058D100107C04129BA7602AFF540CD2F0B506027B
:1058E100C2F0129BA720F0EBF0A3DCE77C04EFC42D
:1058F100540FB4000590E92080D9B401D690EA0094
:1059010080D11280111280EA5389F0438901D28C2F
:10591100D2A9D2AF437DC3306B03129B43306D09D3
:10592100E55C7005128E7EC26D12864D4003029AAF
:10593100F9E57BB57C02802775A0E8A87CE2F9E552
:105941007412847BE91284B5500A0554E554B4A05D
:105951000975540008B810027800887C029A7075A5
:10596100A0F47819E220E003029974781B20E56421
:10597100E270030298E9B4FF22129935307BE910F5
:10598100E612A95077000953016FF70953016F8996
:0E5991005002996FF57EC264029949307BCABC
:10599F00F5F054FCB42822129935F975A0E8A87BCC
:1059AF0030F10574E012992D30F00574F012992D35
:1059BF00E912992D887B02996FA950A7F00953011D
:1059CF006F895002996F7C04A959781BE2FE307BD6
:1059DF0033C3E5592410955A540FB40C007480400A
:1059EF00027481129B90B4801BEE80097819E2300B
:1059FF00E0FC781BE2128534F70953014FDCED8987
:105A0F005902996F029974129935A2E792235000A7
:105A1F00F57E537E7FC264547FB401028013B4308D
:105A2F0002800EB403028009F85300F0B84015D27B
:105A3F00767819E230E0FC30E5030298A8781BE293
:105A4F00F57AD264202320D27C8047F208B8100266
:105A5F007800227819E230E0FC20E504781BE2227E
:105A6F00D0E0D0E00298A8307B2875A0E8A87B741E
:105A7F00EF12992DE57E12992D30640F307607C203
:105A8F007674EF12992DE57A12992D887B74801216
:105A9F009B90107C03029A70E57EB4012FC207E53C
:105AAF007AFE54F0B50614E57F6E54C0700DEEF516
:105ABF00755430C4F576D26F029A6BC27B7575FF41
:105ACF007576FF74AA42C0C2EC029A70B4160C74B9
:105ADF0040B57FE77480129B9080E0B40309E57AAC
:105AEF0090ED00F0029A70B43019E57AC454C0B545
:105AFF007F0EE57A54039092A593457DC57DD26DB7
:105B0F00029A68F95301F0B94024F9C4657F54C073
:105B1F00701AE95403F9307B06B57403857A7975E9
:105B2F0083EA4400F582E57AF01280B78058B40911
:105B3F0024207B028050128EA9F8129B38540FC478
:105B4F004200C074857674128520D074B3E892E752
:105B5F00129B908039B40C07307B02D2EC8027B4B3
:105B6F000208C2EC74AA42C0801CB43119307B14F5
:105B7F00E579540FB40400500BE574D2E212847B24
:105B8F00E41284B58000307B057480129B90306FD7
:105B9F0024E55C6015207209D27290E83FE4F08032
:105BAF001490E83FE0B40200400BC27285595A7559
:105BBF005C00129B6DE5537024E550B551028027B0
:105BCF00A851E6F5560853006F7006865708530024
:105BDF006F8851128B35E553600D75552075A0E810
:105BEF00A855E2F81281C2307302800CE559B55AFC
:105BFF00028005128DC7D273E55C701130731812D5
:105C0F008CEAC273E55C600F755E28C27375A0E8FD
:105C1F00A95EE3F812821F12814C105D14105C060E
:105C2F001075210297EB128EA94490129B90029748
:105C3F00EB129B38F85300070354384844C0129BAB
:105C4F00900297EB7583E8E5744440F582E0547F4A
:105C5F00129B900297EB7583EAE5764400F582E09C
:105C6F0022C26B12855D307B1B128520B3921B20E5
:105C7F001C05301B0F8003201B0AA21B921C74A053
:105C8F0092E0719090E83FE004F0221289EDC26F2C
:105C9F00857674129B38F579128699E57444FCF574
:105CAF0090D27BD2EC128520B3921B921C22C0E0C3
:105CBF0075A0F47819E230E2FCD0E0781BF23001E5
:105CCF00031285522275A0F47819E230E0FC781B9C
:025CDF00E222BF
:025CE1001106AA
:025CE300237F1D
:00000001FF
